:1000000019C033C032C031C030C02FC02EC02DC087
:100010002CC02BC02AC029C028C027C026C025C09C
:1000200024C023C022C021C020C01FC01EC01DC0CC
:100030001CC01BC011241FBECFEFD4E0DEBFCDBF5C
:1000400011E0A0E0B1E0E2E8F0E002C005900D921E
:10005000A030B107D9F711E0A0E0B1E001C01D92D6
:10006000A030B107E1F705D00BC0CACF8FEF8AB936
:1000700008958FEF8AB9589A59985A9A5B98FBCF8E
:02008000FFCFB0
:00000001FF
